:020000040000FA
:100000002E288207003400340034003400341B34BE
:1000100077344034003435346734E03400346A34A3
:10002000CF34C03400349A341D3420340034D534F5
:100030009F34803401341334B234203401344034DA
:100040006F34403401347B34CA3490340134AB34DF
:100050003F3400340134C934C33480348B018316F7
:100060008113FB308500860183120511B220D22056
:10007000051A3B28AB218901FB220808A300FB22BB
:100080000808A400FB220808A500FB220808A60017
:10009000FB2208088C00FB2208088D00FB220808C0
:1000A0008E00FB2208088F0063229122122249222F
:1000B00049220508B30003303305B200B0014030D7
:1000C000AF00B401B7014921B3196828882063281B
:1000D0009D019C019B0101309A00331A7928E83078
:1000E0009A0003309B00792803109A0D9B0D9C0DFC
:1000F0009D0DAF0DB00D031C7428B4188128362156
:100100008328F92011216322912212224922632897
:10011000B41894280430B702D7303707031C92284C
:100120002830B700A0209B280430B707D730370706
:100130000318B701A020632291221222492208004D
:10014000370801208F00B70A370801208E00B70A50
:10015000370801208D00B70A370801208C000330D2
:10016000B70208000B230330860006160B23061285
:100170000330860006160E2306120330860006168C
:100180000E230612023086000616112306122830AE
:10019000CC220830CC220130CC220630CC220C30CC
:1001A000CC2208008030CC225030D0224930D022DE
:1001B0004330D0224530D0224C30D0226730D0227C
:1001C0006530D0226E30D02200238030CC227630B1
:1001D000D0223530D0222E30D0223130D0222D30D6
:1001E000D0223330D0223030D0222030D022002311
:1001F00008001A088C07031C02298D0F02298E0F94
:1002000002298F0A1B088D07031C09298E0F092953
:100210008F0A1C088E07031C0E298F0A1D088F07E2
:100220000800FE300F0703182D2901300F02031CB0
:10023000352936300E0703182D29C9300E02031C4C
:1002400035293C300D0703182D29C3300D02031C3E
:10025000352980300C02031C352980308C00C330D6
:100260008D00C9308E0001308F0008009A099B096B
:100270009C099D099A0F41299B0F41299C0F4129F7
:100280009D0AF9208F1F48298C018D018E018F0155
:100290000800B0014030AF007221B01B5329083074
:1002A000AF070318B00A0508B30003303305B100E7
:1002B000320603194C290310B20D3108B206320878
:1002C0000239B500340603196A293508B40031082B
:1002D000B2004C29B401B21C6F290230B4003108BD
:1002E000B2000800051E7729851980297C29851907
:1002F0007E293918822995293914AA293910AA2961
:10030000B901AA291030BA00051A8B290823BA0BA3
:1003100084290322AA299D010F309C0042309B00B2
:1003200040309A00F9201121A6291030BA00851911
:100330009E290823BA0B97290322AA299D010F3071
:100340009C0042309B0040309A003621632291226B
:1003500012224922080080308C0096308D0098309F
:100360008E0000308F008901FB220808A300FB22C9
:100370000808A400FB220808A500FB220808A60024
:10038000632291221222492249219D019C019B0155
:1003900010309A003319CE2980309A000000B4182A
:1003A000DC299A099B099C099D099A0FDC299B0F5E
:1003B000DC299C0FDC299D0A1A08A307031CE529E8
:1003C000A40FE529A50FE529A60A1B08A407031C0D
:1003D000EC29A50FEC29A60A1C08A507031CF12986
:1003E000A60A1D08A607051EC22989012308880040
:1003F000EE2224088800EE2225088800EE22260836
:100400008800EE220800043089000C088800EE22E3
:100410000D088800EE220E088800EE220F088800E2
:10042000EE2208009501960197019801990120306C
:10043000A0002308A7002408A8002508A900260872
:10044000AA000310271C3B2A0C089607031C2D2A20
:10045000970F2D2A980F2D2A990A0D089707031C2C
:10046000342A980F342A990A0E089807031C392A4F
:10047000990A0F089907990C980C970C960C950CF3
:10048000AA0CA90CA80CA70CA00B212A00309900DB
:100490000800153084000008A2000830A100A20C5A
:1004A000031C562A861506150611592A86110615AB
:1004B0000611A10B4F2A840A1A300402031C4B2A8E
:1004C00086178613080020309E009001910192014A
:1004D0009301940103108C0D8D0D8E0D8F0D03185B
:1004E0000C14900D910D920D930D940D9E03031D10
:1004F0007A2A0800103084008622840A8622840A20
:100500008622840A8622840A86226A2A0330000709
:100510009F009F198000303000079F009F1B8000C4
:1005200008008030CC22130E0F39303ED022130841
:100530000F39303ED022120E0F39303ED022120831
:100540000F39303ED022110E0F39303ED022110823
:100550000F39303ED022100E0F39303ED022100815
:100560000F39303ED02208008601831608308600FD
:10057000831206138616FF30AD0006160608AC007F
:10058000061200000000061600000612AD03031953
:10059000CB2AAC19BD2A0800AB00B8010613D32A38
:1005A000AB0038140617B42286018316003086008B
:1005B00083128612061338180617F03086052B0EA4
:1005C0000F398604061600000612F03086052B0847
:1005D0000F39860406160000061208008316081557
:1005E00055308900AA30890088148818F52A081126
:1005F0008312890A0800831608148312890A0800E6
:1006000005230523052305230800082308230800E4
:10061000FF30AD00162B8030AD00162B4030AD0002
:10062000162B2030AD00162B1030AD00FF30AE0081
:0A063000AE0B182BAD0B162B0800C3
:084000007F007F007F007F00BC
:02400E00F13F80
:10420000C4001D00F3002A0028000100D6000000B1
:10421000000000000000000000000000000000009E
:10422000000000000000000000000000000000008E
:10423000000000000000000000000000000000007E
:10424000000000000000000000000000000000006E
:10425000000000000000000000000000000000005E
:10426000000000000000000000000000000000004E
:10427000000000000000000000000000000000003E
:00000001FF
